:020000040000FA
:04000000FA3060284A
:0800080060188612601C8616C8
:10001000AE00030EAF008312051E15284008E00055
:10002000601C861660188612A214051D1928BC0BC8
:1000300015282830BC000F30A3008B100314851E38
:0E0040000310E00C2F0E8300AE0E2E0E0900F2
:1000C000203084008001840A80300402031C6228EE
:1000D0002830BC008316FF3085055F3086055F3011
:1000E00087058312850186018701103083168E00F3
:1000F0008312703083168F0083120030031799002B
:100100000313003003179A000313003097000030E8
:100110009F00003083169F008312003003179E005B
:100120000313003003179F000313C73083168100A9
:10013000831230309000003092000030831694001B
:10014000831200309400A63083169800831200308A
:1001500083169B0083120030980033308316990079
:100160008312003083168C008312003083168D00BA
:10017000831210308B00B20BBB280130A400810128
:100180008E018F010B118B100B108C128C018D01C5
:100190008B1764000B19D720E620C92848085002A5
:1001A000031DD4285008C0004808D00008000B11D7
:1001B000A40B08000430A400A3080319E228861346
:1001C000A303080006098039860008000608A0007D
:1001D0000708A1002118F1280130A5070318F62807
:1001E000FD280130A502031CFA28FD28FF30A500D8
:1001F0004814FD28A5014810FD28A1180429013044
:10020000A6070318092910290130A602031C0D298D
:100210001029FF30A600C8141029A601C810102903
:10022000211917290130A70703181C292329013098
:10023000A702031C20292329FF30A70048152329E2
:10024000A70148112329201A2A290130A8070318D9
:100250002F2936290130A802031C33293629FF3003
:10026000A800C8153629A801C8113629211A3D2928
:100270000130A9070318422949290130A902031CAA
:1002800046294929FF30A90048164929A9014812E1
:100290004929201B50290130AA07031855295C2938
:1002A0000130AA02031C59295C29FF30AA00C81694
:1002B0005C29AA01C8125C29211B63290130AB0704
:1002C000031868296F290130AB02031C6C296F29C0
:1002D000FF30AB0048176F29AB0148136F29A119F4
:1002E00076290130AC0703187B2982290130AC0242
:1002F000031C7F298229FF30AC00C8178229AC017A
:10030000C8138229CE2008000708803A8700080019
:100310000708203A870008000608803A860008008F
:084000000800000001000200AD
:02400E00CC03E1
:00000001FF
